:100000006F282C08A0002D08A100A201A301082838
:10001000092864008C1A1F28FF30A207031CA307BD
:10002000031CA007031CA107031C6A28220F072832
:10003000230F08283230A2000030A30009281A0834
:1000400003146A28A501A400B3172730A3001030B9
:1000500035200330A300E8303520A301643035207B
:10006000A3010A30352024084028A2002508A10059
:100070002408A0004E202008031DB313B31B080062
:10008000303E64000C1E4128990003146A2883172F
:100090008001840AFF3E031D48286A28A501A401A7
:1000A0001030A600210DA40DA50D2208A4022308DE
:1000B000031C230FA502031864282208A4072308A1
:1000C0000318230FA5070310A00DA10DA60B52289E
:1000D00020086A2883130313831264000800831620
:1000E0000C30990024309800831290309800203012
:1000F000840060308A014820A030840050308A019A
:1001000048201030840060308A01472090308400FD
:1001100060308A014720A03087008316A030870016
:100120008501831285018316810183120D308A01B6
:10013000412043308A01412048308A0141204F301C
:100140008A0141204F308A01412053308A014120E9
:1001500045308A01412020308A0141204D308A01FA
:1001600041204F308A01412044308A0141204530EE
:100170008A0141203A308A0141200A308A01412017
:100180000D308A01412001308A01222029308A0164
:10019000412020308A0141204F308A0141205030D7
:1001A0008A01412045308A0141204E308A01412098
:1001B0000A308A0141200D308A01412002308A0133
:1001C000222029308A01412020308A0141204130FB
:1001D0008A01412055308A01412054308A01412052
:1001E0004F308A0141200A308A0141200D308A01B6
:1001F000412003308A01222029308A014120203009
:100200008A01412045308A01412058308A0141202D
:1002100049308A01412054308A0141200A308A0144
:1002200041200D308A01412004308A0122202930EA
:100230008A01412020308A0141204F308A0141202B
:1002400046308A01412046308A0141200A308A0125
:1002500041200D308A014120F430AC000130AD0066
:100260008A0101208A110A12031C2C29B80030309F
:10027000B8026400053038028A110A1203184F29A7
:100280003808043C8A110A12031C4F2901308A00E5
:10029000380882078A29C529F529262A582A0D30C7
:1002A0008A01412045308A01412052308A01412093
:1002B00052308A0141204F308A01412052308A0158
:1002C00041200A308A0141200D308A0141205430FA
:1002D0008A01412052308A01412059308A0141204F
:1002E00020308A01412041308A01412047308A0173
:1002F000412041308A01412049308A0141204E305D
:100300008A0141200A308A0141200D308A014120B2
:100310008A0196280D308A01412045308A0141200A
:1003200052308A01412052308A0141204F308A01E7
:10033000412052308A0141200A308A0141200D308B
:100340008A01412054308A01412052308A014120E3
:1003500059308A01412020308A01412041308A01F0
:10036000412047308A01412041308A0141204930F3
:100370008A0141204E308A0141200A308A01412001
:100380000D308A0141208A0196280D308A014120D2
:100390004F308A01412050308A01412045308A0186
:1003A00041204E308A01412020308A0141204D30C9
:1003B0008A0141204F308A01412044308A01412086
:1003C00045308A01412020308A0141204F308A0186
:1003D00041204E308A0141200A308A0141200D30EF
:1003E0008A01412005148A0196280D308A01412096
:1003F00041308A01412055308A01412054308A0120
:1004000041204F308A01412020308A0141204D3067
:100410008A0141204F308A01412044308A01412025
:1004200045308A01412020308A0141204F308A0125
:1004300041204E308A0141200A308A0141200D308E
:100440008A014120051085148A0196280D308A0101
:10045000412045308A01412058308A0141204930ED
:100460008A01412054308A01412020308A014120F4
:100470004D308A0141204F308A01412044308A01A9
:10048000412045308A01412020308A0141204F30EF
:100490008A0141204E308A0141200A308A014120E0
:1004A0000D308A0141200510851005158A01962816
:1004B0000D308A0141204F308A01412046308A01A7
:1004C000412046308A01412020308A0141204D30B0
:1004D0008A0141204F308A01412044308A01412065
:1004E00045308A01412020308A0141204F308A0165
:1004F00041204E308A0141200A308A0141200D30CE
:100500008A01412005108510051185158A0196285C
:040510008A0196289E
:02400E00723FFF
:00000001FF
